:10000000F8C000002CC1000010C100000EC10000AB
:100010000CC100000AC1000008C1000006C10000B8
:1000200004C1000002C1000000C10000FEC00000C9
:10003000FCC00000FAC00000F8C00000F6C00000DC
:100040000C949B11F2C00000F0C00000EEC0000054
:10005000ECC00000EAC00000E8C00000E6C00000FC
:10006000E4C00000E2C00000130B1C0B190B180BBE
:10007000170B160B150B140B1D0B1D0B1D0B1D0B5E
:100080001D0B1D0B1D0B1D0B1A0B1D0B1D0B1D0B33
:100090001D0B1D0B1D0B1D0B1B0B0902220001016B
:1000A0000080320904000001030000000921010161
:1000B00000012272000705810308000A12011001E5
:1000C00000000008C410C0820001010200012A03E0
:1000D0005500530042002000520065007400720079
:1000E0006F00500061006400200041006400610066
:1000F00070007400650072002A03770077007700B3
:100100002E006200720075006E006F0066007200C3
:10011000650069007400610073002E0063006F00C9
:100120006D000403090405010905A101150025015D
:10013000350045017501950D05091901290D81024B
:100140009503810105012507463B0175049501656D
:10015000140939814265009501810126FF0046FF9F
:1001600000093009310932093509367508950581CC
:10017000020600FF09200921092209230924092573
:100180000926092709280929092A092B950C810222
:100190000A21269508B102C00000000700020100F4
:1001A0000003040600000000000000000102040833
:1001B00010204080010204081020010204081020D1
:1001C00004040404040404040202020202020303FD
:1001D00003030303000000002300260029000000A1
:1001E0000000250028002B0000000000240027004C
:1001F0002A0011241FBECFEFD4E0DEBFCDBF11E037
:10020000A0E0B1E0E0EDF5E202C005900D92A0346F
:10021000B107D9F721E0A0E4B1E001C01D92AF3FE2
:10022000B207E1F770D20C94E612EACEA82FB92FEC
:1002300080E090E041E050EA609530E009C02D9107
:1002400082279795879510F084279527305EC8F30D
:100250006F5FA8F30895EADF8D939D930895CF9380
:10026000CFB7CF93DF93C3954C9BE9F74C9B0BC063
:100270004C9B09C04C9B07C04C9B05C04C9B03C0CA
:100280004C9B01C08BC06F93C091E201DD27C75129
:10029000DE4F2F9365E54C9B03C02F916F91E6CF06
:1002A0000F931F934F9320E040E15F9309B10471D6
:1002B00004FB27F93F9350E03BE039C014714064E0
:1002C0002F77012F5F5F1EC0406819B114712F771F
:1002D00052501FC0406409B12F770471D1F15F5FA4
:1002E00000C023C0406219B12F77147191F15F5F94
:1002F00000C025C004711027515012F45D5F00004A
:10030000115027952C3F19B1C8F6147101270150DF
:1003100027952C3FC8F64227499309B1047110274D
:100320004F73115027952C3FA8F64695469519B165
:10033000147179F00127015027952C3F98F66B5ADC
:1003400060F3315009B1B0F600C011E01CBB0027CA
:1003500019C03B503195C31BD04011E01CBB088134
:10036000033C09F10B34F9F02091E0011981110FE0
:100370001213EDCF4A81441F093651F10D3211F0AD
:10038000013E29F70093E7013F915F914F911F9143
:100390000F912F916F91CCB3C0FD65CFDF91CF91BD
:1003A000CFBFCF9118952091E701222369F31091D7
:1003B000E501112391F5343092F13093E50120935A
:1003C000E1011091E2013BE0311B3093E20127C0D3
:1003D0000091E50101300CF50AE54F7049F43091C8
:1003E000050134FD1DC000930501C9ECD1E01CC01E
:1003F0003091D40134FD14C00093D401C5EDD1E097
:1004000013C0052710E000C000000BB91AC0052773
:1004100010E0221F1DC010E021C04AE502C032EDED
:10042000432FC4E1D0E032E01AB114615C9A0BB101
:100430001AB954E120E865E320FF05270BB9279599
:1004400017951C3FF0F66695B8F7B1F720FF052722
:100450000BB9279517951C3FD0F62795179517FFD1
:10046000052700001C3F0BB9B0F629913A9519F702
:100470000B7E1091E601110FC651D0400BB911F05F
:100480001093E00111E01CBB00611AB11B7E402FEC
:100490004B7E54E05A95F1F70BB91AB94BB974CFAA
:1004A000CF93C62F2091D40124FF07C02091D501FE
:1004B00038E823272093D50103C02AE52093D401EF
:1004C000DC01E6EDF1E09C2F9E0F8D918193892F49
:1004D0008E1B1816D4F36C2F86ED91E0BCDECC5F3A
:1004E000C093D401CF910895CF93DF938091E5011C
:1004F000835087FDA4C09091E2012091E1012D324B
:1005000009F09BC0883009F098C0CCE0D0E0C91B4E
:10051000D109C751DE4F83EC8093C9018AE58093EE
:100520000501109240018881807621F0CE010E9461
:10053000900B7AC09A811092D2018981811106C0F4
:100540001092D30122ED31E082E06AC0853019F4C7
:100550009093E60162C0863009F049C08B818130FA
:1005600041F48CEB90E09093E4018093E30182E10D
:100570003AC0823041F48AE990E09093E40180939C
:10058000E30182E230C08330C9F4911108C082E2F5
:1005900091E09093E4018093E30184E024C09130E2
:1005A00019F488EF90E004C09230E1F48EEC90E012
:1005B0009093E4018093E3018AE215C0813241F413
:1005C0008CEA90E09093E4018093E30189E00BC012
:1005D000823241F486E291E09093E4018093E3015A
:1005E00082E701C080E090E4909340011DC0883014
:1005F00069F0893019F49093E8010FC08A3049F00E
:100600008B3059F48BE48093D50107C028EE31E09C
:1006100002C022ED31E081E003C022ED31E080E054
:100620003093E4012093E3019F81911104C09E81E6
:10063000981708F4892F809304011092E5018091A6
:10064000050184FF46C0809104018F3F09F441C039
:10065000C82F893008F0C8E08C1B8093040180917A
:10066000C90198E889278093C901CC2331F12091F1
:10067000E3013091E4018091400186FF0BC0AAECB8
:10068000B1E0F9018C2F8A0F94919D9331968A13D2
:10069000FBCF09C0D901EAECF1E08C2F8E0F9D91C0
:1006A00091938E13FCCF8FEF8C0F90E00196820F09
:1006B000931F9093E4018093E3016C2F8AEC91E007
:1006C000CADDCC5FCC3019F08FEF80930401C0936A
:1006D000050184E199B1947131F48150D9F71092F8
:1006E000E6011092E001DF91CF910895E9E6F0E094
:1006F000808182608083E89A8BE48093D5018AE5CB
:100700008093D40108950E94EF11A5D083D7FECF26
:10071000CF92DF92EF92FF920F931F93CF93DF93CD
:1007200060E086E00E941C1161E086E00E943C11BE
:1007300060E088E00E941C1161E088E00E943C11AA
:1007400060E089E00E941C1161E089E00E943C1198
:1007500060E08AE00E941C1161E08AE00E943C1186
:1007600060E08BE00E941C1161E08BE00E943C1174
:1007700060E08CE00E941C1161E08CE00E943C1162
:100780008CE00E947311892B09F057C086E00E940B
:100790007311892B19F4C0E1D0E002C0C0E0D0E0B1
:1007A00088E00E947311892B19F408E010E002C060
:1007B00000E010E089E00E9473116C018AE00E9461
:1007C00073117C018BE00E9473119801282B392B47
:1007D0002C2B3D2BCC0CDD1CCC0CDD1C2C293D29FD
:1007E000EE0CFF1C2E293F29C90143E09595879502
:1007F0004A95E1F783709927892BD9F02B31310580
:1008000079F03CF42F303105D9F02731310541F032
:100810000DC02C31310539F02F31310589F006C07A
:1008200087E190E00FC084E090E00CC087E090E0AA
:1008300009C0C9018770992705C08FEF9FEF02C0DB
:100840008FE090E0DF91CF911F910F91FF90EF909B
:10085000DF90CF90089581E007C789D7C0E8DFEF28
:1008600039D794D7C0934501C093460182FF03C096
:100870001092450103C083FDD093450180FF03C062
:100880001092460103C081FDD093460131E086FFFE
:1008900030E02091420130FB20F920934201217089
:1008A00021952093510131E084FF30E020914201F5
:1008B00030FB21F920934201269521702195209348
:1008C000500131E085FF30E02091420130FB22F9F8
:1008D0002093420122FB222720F9219520934F01EA
:1008E00031E092FF30E02091420130FB24F9209367
:1008F00042012295217021952093520131E091FF10
:1009000030E02091420130FB23F92093420123FB88
:10091000222720F9219520934E0131E090FF30E00D
:100920002091420130FB25F92093420125FB22272B
:1009300020F921952093530131E093FF30E020917D
:10094000430130FB20F92093430131E087FF30E081
:100950002091430130FB21F92093430181789927AD
:1009600021E08138910509F020E08091430120FBCE
:1009700084F980934301B0D673CF4DE050E067E037
:1009800070E086E090E00E940F0EC0E8DFEFA2D694
:1009900080E190E00E942D0EC093450180FF03C0CE
:1009A0001092460107C081FD03C0C093460102C0FA
:1009B000D093460182FF03C01092450103C083FD1E
:1009C000D093450131E084FF30E02091420130FBBB
:1009D00020F920934201217021952093510131E0AB
:1009E00085FF30E02091420130FB21F92093420144
:1009F0002695217021952093500131E086FF30E04B
:100A00002091420130FB23F92093420123FB22274E
:100A100020F9219520934E0131E087FF30E02091AD
:100A2000420130FB22F92093420122FB222720F9C8
:100A3000219520934F0131E090FF30E02091420159
:100A400030FB24F9209342012295217021952093B7
:100A5000520131E091FF30E02091420130FB25F955
:100A60002093420125FB222720F921952093530151
:100A700031E092FF30E02091420130FB26F92093D3
:100A8000420126FB222720F921952093540131E0D1
:100A900093FF30E02091420130FB27F9209342017F
:100AA000220F220B2093550131E094FF30E020917A
:100AB000430130FB20F92093430131E095FF30E002
:100AC0002091430130FB21F92093430121E096FF5F
:100AD00020E08091430120FB82F9991F9927991FFB
:100AE00090FB84F980934301F7D551CF47E050E064
:100AF00066E070E085E090E00E940F0EC0E8DFEF56
:100B0000E9D588E090E00E942D0EC0934501C09386
:100B1000460186FF03C01092450103C087FDD093B4
:100B2000450184FF03C01092460103C085FDD093A8
:100B3000460131E081FF30E02091420130FB20F995
:100B400020934201217021952093510131E080FFD3
:100B500030E02091420130FB21F92093420126959B
:100B6000217021952093500131E082FF30E02091E7
:100B7000430130FB20F92093430131E083FF30E053
:100B80002091430130FB21F9209343018C70992778
:100B900021E00C9709F020E08091430120FB84F9CB
:100BA0008093430199D5ACCF47E050E066E070E018
:100BB00085E090E00E940F0EC0E8DFEF8BD580E16A
:100BC00090E00E942D0EC0934501C093460186FF20
:100BD00003C01092450103C087FDD093450184FFF7
:100BE00003C01092460103C085FDD093460131E059
:100BF00081FF30E02091420130FB20F92093420137
:100C0000217021952093510131E080FF30E0209147
:100C1000420130FB21F92093420126952170219554
:100C20002093500131E090FF30E02091420130FBF1
:100C300022F92093420122FB222720F921952093BB
:100C40004F0131E092FF30E02091420130FB24F966
:100C5000209342012295217021952093520131E089
:100C600091FF30E02091420130FB23F920934201B3
:100C700023FB222720F9219520934E0131E093FF99
:100C800030E02091420130FB25F92093420125FB01
:100C9000222720F921952093530131E082FF30E093
:100CA0002091430130FB20F92093430131E083FF81
:100CB00030E02091430130FB21F9209343018C70F7
:100CC000992721E00C9709F020E08091430120FB57
:100CD00084F98093430100D571CF81E00E94040F15
:100CE000892B39F0F7D480E197E20E94E511F4D422
:100CF000F4CFC0E8DFEFEED40E94E80E0E94970F19
:100D000081112DC0C0934701C093480180E890E055
:100D10000E94850F882319F0109245010BC080E2D4
:100D200090E00E94850F882319F0D093450102C0FE
:100D3000C093450180E190E00E94850F882319F05F
:100D4000109246014BC080E490E00E94850F8823FA
:100D500019F0D093460142C0C09346013FC087E0DE
:100D600090E00E94920F8093450188E090E00E94FD
:100D7000920F8093460185E090E00E94920F80934D
:100D8000470186E090E00E94920F8093480180E145
:100D900090E00E94850FF82E80E490E00E94850F7D
:100DA000082F80E890E00E94850F182F80E290E0E5
:100DB0000E94850F98E0F99EA001112494E0099FFC
:100DC00090011124242B282B812F880F822BE82FB0
:100DD000F0E0EA5FFE4F80818093440180E090E87C
:100DE0000E94850F9091420180FB90F990934201FF
:100DF000917091959093510180E090E40E94850F4D
:100E00009091420180FB91F99093420196959170E7
:100E100091959093500180E090E20E94850F90910F
:100E2000420180FB92F99093420192FB992790F93D
:100E3000919590934F0180E094E00E94850F9091EE
:100E4000420180FB94F990934201929591709195A3
:100E50009093520180E091E00E94850F90914201B1
:100E600080FB96F99093420196FB992790F9919512
:100E70009093540180E090E10E94850F909142018F
:100E800080FB93F99093420193FB992790F99195F8
:100E900090934E0180E098E00E94850F909142016E
:100EA00080FB95F99093420195FB992790F99195D4
:100EB0009093530180E092E00E94850F909142014F
:100EC00080FB97F990934201990F990B90935501EC
:100ED00082E090E00E94850F9091430180FB92F99F
:100EE0009093430184E090E00E94850F909143012C
:100EF00080FB93F99093430181E090E00E94850F7D
:100F00009091430180FB90F99093430188E090E039
:100F1000FCD79091430180FB91F99093430181E0CC
:100F200090E0F3D7882331F088E090E0EED791E0AD
:100F3000811101C090E08091430190FB84F980937E
:100F40004301CAD3D8CE9AD5811107C0C3D380E15B
:100F500097E20E94E511C0D3F6CF99249A94BAD3B0
:100F6000C0D5EC01898183FD02C0E0E001C0E8E06A
:100F700082FD02C020E001C024E080FD02C090E0BC
:100F800001C092E031E081FF30E0E32BE22BE92B5E
:100F9000FF27E7FDF095EA5FFE4F808180934401D3
:100FA000888191E083FF90E08091420190FB80F97D
:100FB000809342018170819580935101888191E0F5
:100FC00081FF90E08091420190FB81F98093420182
:100FD00086958170819580935001888191E082FF90
:100FE00090E08091420190FB83F98093420183FB62
:100FF000882780F9819580934E01888191E080FF58
:1010000090E08091420190FB82F98093420182FB43
:10101000882780F9819580934F01888191E084FF32
:1010200090E08091430190FB81F980934301898195
:1010300091E086FF90E08091420190FB84F98093DB
:10104000420182958170819580935201898191E05E
:1010500085FF90E08091420190FB85F980934201E9
:1010600085FB882780F9819580935301898191E0E0
:1010700084FF90E08091420190FB86F980934201C9
:1010800086FB882780F9819580935401898183FFAD
:1010900004C098819295917001C090E080914301C5
:1010A00090FB84F9809343016A8170E080E090E0D6
:1010B0001F921F921F929F92A12CB12C65011FEDD0
:1010C000E12EF12C00E010E020E230E040E050E0C2
:1010D0000E942A12609345016B81609570E080E068
:1010E00090E01F921F921F929F9220E230E040E01A
:1010F00050E00E942A12609346016C8170E080E00B
:1011000090E01F921F921F929F9220E230E040E0F9
:1011100050E00E942A12609347016D81609570E053
:1011200080E090E01F921F921F929F9220E230E099
:1011300040E050E00E942A12609348018F8186951A
:1011400080589E819695891B80934901C5D288E875
:1011500093E10E94E5118DB79EB740960FB6F894C3
:101160009EBF0FBE8DBFFBCE89D4811107C0B2D206
:1011700080E197E20E94E511AFD2F6CF99249A94CC
:10118000F0E88F2EA7D2FFD4EC01888183FD02C046
:10119000E0E001C0E8E082FD02C020E001C024E000
:1011A00081FD02C090E001C092E031E080FF30E0BC
:1011B000E32BE22BE92BFF27E7FDF095EA5FFE4FDB
:1011C000808180934401888191E086FF90E0809146
:1011D000420190FB80F98093420181708195809358
:1011E00051018881982F991F9927991F8091420159
:1011F00090FB81F98093420186958170819580935F
:101200005001888191E084FF90E08091430190FB40
:1012100081F980934301898191E085FF90E080917D
:10122000420190FB84F980934201829581708195FF
:1012300080935201898191E084FF90E08091420186
:1012400090FB85F98093420185FB882780F9819581
:1012500080935301888191E085FF90E08091420165
:1012600090FB86F98093420186FB882780F981955F
:10127000809354018881887191E0883109F090E071
:101280008091430190FB84F9809343016A81605807
:10129000609345018B81805880958093460170E072
:1012A00080E090E01F921F921F929F92A12CB12C80
:1012B00065011FEDE12EF12C00E010E020E230E0AE
:1012C00040E050E00E942A1260934501609146017F
:1012D00070E080E090E01F921F921F929F9220E2A8
:1012E00030E040E050E00E942A1260934601809274
:1012F00047018092480189812DB73EB7285F3F4F53
:101300000FB6F8943EBF0FBE2DBF83FF03C01092EF
:10131000480103C082FD90924801898181FF03C08A
:101320001092470103C080FD90924701D5D12ACF8A
:1013300047E050E066E070E085E090E070D4C0E8FF
:10134000DFEFC8D180E190E088D4C0934501C0931D
:10135000460181FF03C01092450103C093FDD09365
:10136000450182FF03C01092460103C094FDD09353
:10137000460120914201392F331F3327331F30FBA1
:1013800020F920934201217021952093510131E0F1
:1013900080FF30E02091420130FB21F9209342018F
:1013A0002695217021952093500131E092FF30E085
:1013B0002091420130FB22F92093420122FB222797
:1013C00020F9219520934F0131E091FF30E02091E9
:1013D000420130FB23F92093420123FB222720F90D
:1013E000219520934E0131E090FF30E020914301A0
:1013F00030FB20F92093430131E096FF30E020914B
:10140000430130FB21F9209343018827917421E0A7
:101410008115914409F020E08091430120FB84F97B
:101420008093430159D18DCF92D5C0E8DFEF52D1DF
:101430009BD5C0934501C093460192FF03C0109213
:10144000450103C093FDD093450190FF03C0109266
:10145000460103C091FDD093460131E086FF30E0A4
:101460002091420130FB20F9209342012170219507
:101470002093510131E084FF30E02091420130FBA4
:1014800021F9209342012695217021952093500146
:1014900031E085FF30E02091420130FB22F92093BA
:1014A000420122FB222720F9219520934F0131E0B0
:1014B00082FF30E02091420130FB24F92093420169
:1014C0002295217021952093520131E081FF30E077
:1014D0002091420130FB23F92093420123FB222774
:1014E00020F9219520934E0131E080FF30E02091DA
:1014F000420130FB25F92093420125FB222720F9E8
:1015000021952093530131E094FF30E02091420176
:1015100030FB26F92093420126FB222720F9219552
:101520002093540131E083FF30E02091420130FBF1
:1015300027F920934201220F220B2093550131E01D
:1015400087FF30E02091430130FB21F920934301D4
:101550008078917021E08038914009F020E08091FE
:10156000430120FB84F980934301B6D060CF91D52D
:10157000C0E8DFEFAFD09AD5C0934501C0934601D4
:1015800083FF03C01092450103C081FDD093450144
:1015900080FF03C01092460103C082FDD093460134
:1015A00021E085FF20E09091420120FB90F990938B
:1015B0004201917091959093510121E084FF20E0C8
:1015C0009091420120FB91F9909342019695917080
:1015D00091959093500121E087FF20E09091430185
:1015E00020FB91F99093430191E086FF90E0809178
:1015F000430190FB80F980934301837091E0833035
:1016000009F090E08091430190FB84F980934301BD
:1016100063D0B0CF7DD801968931910570F48C5C90
:101620009F4FFC0192C7A9D961DABEDA56DB8BDC89
:101630009BDD7EDEF9DE9BDFFFCF0FD984E1E2E4A4
:10164000F1E0DF011D928A95E9F788E0809344017B
:1016500080E8809345018093460180934701809301
:101660004801809349010895CF93DF931F92CDB72E
:10167000DEB790916E009E7F90936E008983DEDFCF
:101680008981882361F02FE088E190E00FB6F8941B
:10169000A895809360000FBE2093600008C088E189
:1016A0000FB6F89480936000109260000FBE1ED8B1
:1016B000549A80E0815041F0A895EFE9FFE031971E
:1016C000F1F700C00000F6CF549878940F90DF91A6
:1016D000CF910895A89508958091D40184FD03C009
:1016E0000E947402F9CF68E082E491E00E94500207
:1016F0008091D40184FD03C00E947402F9CF68E098
:101700008AE491E00E9450028091D40184FD03C0DC
:101710000E947402F9CF64E082E591E00C945002DB
:10172000FC0180818076803201F58181813071F405
:1017300083818330D1F48281811117C086E191E0E9
:101740009093E4018093E30188E00895823041F4AE
:1017500081E491E09093E4018093E30181E00895B6
:101760008A3019F483818093410180E0089555986F
:101770005698579820982198229A23985D9A5E9AB5
:101780005F9A289A299A2A9A2B9A0895EF92FF92A3
:101790000F931F93CF93DF932A9A8EE090E015D694
:1017A00089B182958695877091E089278170C82FCD
:1017B00080E0D82F4E9903C082E090E002C080E024
:1017C00090E0C82BD92B4F9903C084E090E002C071
:1017D00080E090E0C82BD92B189903C048E050E076
:1017E00002C040E050E0C42BD52B199903C020E182
:1017F00030E002C020E030E0C22BD32B1B9903C0A5
:1018000020E230E002C020E030E0C22BD32B2A9847
:101810008EE090E0DAD54F9902C0189B02C0CE014D
:1018200060C0199B25C080E090E08C2B9D2B1B99FC
:1018300003C020E830E002C020E030E07C01E22A72
:10184000F32A2A9A8EE090E0C0D52A988EE090E0A4
:10185000BCD54D9906C04E9904C04F9902C0189B43
:101860000AC0C0E0D0E09C2F88278E299F2939C06C
:1018700080E490E0DACF2A9A8EE090E0A6D589B194
:1018800082958695877091E08927082F017010E076
:101890004E9B24C020E030E0E901C02BD12B4F99B2
:1018A00003C084E090E002C080E090E0C82BD92B18
:1018B000189903C048E050E002C040E050E0C42B5B
:1018C000D52B2A988EE090E080D52A9A8EE090E081
:1018D0007CD52A9880ED97E078D5C5CF22E030E01E
:1018E000DBCFDF91CF911F910F91FF90EF90089583
:1018F000559A20E8FC01408142235D9830E009F4CC
:1019000040C00000000000000000000000000000D7
:101910005D9A35952795211112C0019661500000FE
:1019200000000000000000000000000000000000B7
:101930000000000000000000000020E814C00000CB
:101940000000000000000000000000000000000097
:101950000000000000000000000000000000000087
:101960000000000000000000000000000000000077
:101970000000000000000000000000000000000067
:1019800040C0000000000000000000000000000057
:10199000000000000000000000003595279521118F
:1019A00012C001966150000000000000000000001D
:1019B0000000000000000000000000000000000027
:1019C000000020E813C0000000000000000000003C
:1019D0000000000000000000000000000000000007
:1019E0000000000000000000000000005D9A000000
:1019F00000000000000000000000000000000000E7
:101A00000000611177CF000000005D980000000029
:101A100000000000000000000000000000000000C6
:101A200000000000000000005D9A089555985D9A3E
:101A3000E2E6F1E08E0F4D99FECF000000000000BD
:101A40000000000000000000000000000000000096
:101A50000000000000000000000000000000000086
:101A60000000000000000000000099B19072919306
:101A70008E1719F04D9BFECFDECF08951F93CF93A5
:101A8000DF931F92CDB7DEB71982E2E6F1E0119243
:101A900081E0E23AF807D9F7EAE5F1E0119281E056
:101AA000E236F807D9F710925601109257011092BA
:101AB000580110925901F89461E0CE01019618DFA7
:101AC00055985D9A10E44D9B02C01150E1F778944F
:101AD00084EF91E07AD4812F0F90DF91CF911F9105
:101AE00008951F93CF93DF9300D01F92CDB7DEB739
:101AF00080E4898383E08A831B82F89463E0CE01CB
:101B00000196F6DE80E492DF7894EAE5F1E042E6C1
:101B100051E087E090E061E070E020E030E0DA0141
:101B2000A20FB31FAC91AA2351F01081DB01082E44
:101B300001C0AA0F0A94EAF71A2B10830AC0DB012E
:101B4000082E01C0AA0F0A94EAF7A095B081BA2323
:101B5000B083019797FF02C087E090E02F5F3F4F6F
:101B600028303105E1F63196485F5F4F21E0E236DB
:101B7000F20799F68AE591E00F900F900F90DF91B0
:101B8000CF911F9108951F93CF93DF931F92CDB7ED
:101B9000DEB781E08983F89461E0CE010196A8DE8A
:101BA00080E244DF7894E6E5F1E042E651E087E048
:101BB00090E061E070E020E030E0DA01A20FB31FB6
:101BC000AC91AA2351F01081DB01082E01C0AA0FAD
:101BD0000A94EAF71A2B10830AC0DB01082E01C011
:101BE000AA0F0A94EAF7A095B081BA23B0830197AF
:101BF00097FF02C087E090E02F5F3F4F283031050C
:101C0000E1F63196485F5F4F21E0EA35F20799F639
:101C100086E591E00F90DF91CF911F910895CF93CA
:101C2000DF938093A6019093A7017093A501609321
:101C3000A4015093A3014093A20161E0FDD261E0B1
:101C40008091A401F9D2C2EAD1E060E08881F4D2A7
:101C500061E08881DF91CF910FC3EF92FF920F93E4
:101C60001F93CF93DF937C0160E08091A40104D3A4
:101C700060E08091A60100D361E08091A401FCD2D4
:101C800081E090E0A2D360E08091A401F5D2809140
:101C9000A20129D38C01C1E0D0E0CE15DF05C4F448
:101CA00061E08091A601E8D281E090E08ED360E00F
:101CB0008091A601E1D28091A20115D30C2E02C021
:101CC000880F991F0A94E2F7082B192B2196E5CF6C
:101CD000C80180959095DF91CF911F910F91FF9052
:101CE000EF900895CF92DF92EF92FF920F931F93A0
:101CF000CF93DF93C0E0D0E0D12C082F10E0EE248A
:101D0000E394F12C2898CC2EA8010C2E02C05595F6
:101D100047950A94E2F740FF02C05E9A01C05E98C0
:101D200084E190E052D3289A4D9B07C097010C2C78
:101D300001C0220F0A94EAF7D22A84E190E045D349
:101D40002196C830D105F1F6289A83E090E03DD382
:101D50008D2DDF91CF911F910F91FF90EF90DF902C
:101D6000CF900895EF92FF920F931F93CF93DF933D
:101D7000182FF92E062F8091A901882309F0F894D5
:101D80005F985E9A289A86E090E01FD3E12EC12FDB
:101D9000DF2D8C2F8E19801720F48881A3DF899383
:101DA000F8CF5F9A8091A901882309F07894209157
:101DB0001E0188EE93E0AC01249FC001259F900D89
:101DC0001124DF91CF911F910F91FF90EF90FDC2F1
:101DD00081E08093AA0182E48093AB0120911E01EF
:101DE00088EE93E0AC01249FC001259F900D112443
:101DF000ECD2ECEAF1E0119251E0EF3BF507D9F7B4
:101E000065E18AEA91E0AECFFF920F931F93CF93E3
:101E1000DF93CDB7DEB7A0970FB6F894DEBF0FBE45
:101E2000CDBF8093A90155985D9A209A579A569AEA
:101E3000289A5E9ACDDF8091AB01813429F08337F7
:101E400019F0893709F050C081E080931E0103E04A
:101E500095E0F92E19E0EFE1F1E0DE015C968F2DBF
:101E600001900D928A95E1F765E0CE014C967ADFFC
:101E7000E4E2F1E0DE015396812F01900D928A9504
:101E8000E1F769E0CE0143966DDF8E898093BF0153
:101E9000EDE2F1E0DE011A96812F01900D928A9514
:101EA000E1F769E0CE010A965DDFE6E3F1E0DE01ED
:101EB0001196812F01900D928A95E1F769E0CE018C
:101EC000019650DF85DF8091AB01833721F481E0FB
:101ED0008093A8010CC080911E018F5F80931E012A
:101EE000015009F0B8CF03C081E090E002C080E06B
:101EF00090E0A0960FB6F894DEBF0FBECDBFDF9185
:101F0000CF911F910F91FF9008952091AD013091D5
:101F1000AE01209530952823392381E0232B09F445
:101F200080E0089586559E4FFC0180810895809140
:101F3000BF01833041F09091A801911104C081301C
:101F400021F482E0089581E0089580E00895559895
:101F5000569822982398579A219A5D9A5E9A2A9ABF
:101F60002B9A5F9A299A08950F931F93CF93DF932B
:101F70005F9A299A84E090E028D21A9903C000E081
:101F800010E102C000E010E05F98299884E090E042
:101F90001CD289B1829586958695837091E08927B8
:101FA0008170C82F80E0D82FC02BD12B4D9903C052
:101FB00042E050E002C040E050E0C42BD52B1B991A
:101FC00003C044E050E002C040E050E04C2B5D2BE9
:101FD0001A9903C028E030E002C020E030E0EA01B6
:101FE000C22BD32B5F9A299884E090E0EED14E99D2
:101FF00003C080E190E002C080E090E0C82BD92BC4
:102000004D9903C040E250E002C040E050E0C42BD4
:10201000D52B1B9903C020E430E002C020E030E063
:10202000C22BD32B1A9903C080E890E002C080E055
:1020300090E0C82BD92B5F98299A84E090E0C5D115
:102040004E9903C040E051E002C040E050E04C2B0C
:102050005D2B4D9903C020E032E002C020E030E06B
:10206000242B352B1B9903C080E094E002C080E054
:1020700090E0822B932B1A9903C020E038E002C035
:1020800020E030E0822B932BDF91CF911F910F91B5
:10209000089555985D9A57985F9A2098289A2198A4
:1020A000299A229A2A9A239A2B980895DF92EF92DE
:1020B000FF920F931F93CF93DF932A9A2B9882E07E
:1020C000E82EF12CC0E0D0E0DD24D3942B9881E001
:1020D00090E07BD14D993DC04F993BC0189939C0D4
:1020E000199937C02A9881E090E06FD14D9B2EC09E
:1020F00080E090E0C82BD92B4F9903C020E032E05C
:1021000002C020E030E0C22BD32B189903C020E09E
:1021100034E002C020E030E0C22BD32B199903C079
:1021200020E038E002C020E030E0C22BD32B2A9A16
:102130002B9A81E0E81AF10849F6CE01DF91CF91A0
:102140001F910F91FF90EF90DF90089580E091E054
:10215000D1CF89B18295869587708D25082F017022
:1021600010E00C2B1D2B4F9B3BC080E090E0E80162
:10217000C82BD92B189903C024E030E002C020E01E
:1021800030E0C22BD32B199903C028E030E002C005
:1021900020E030E0C22BD32B2A9881E090E015D1CB
:1021A0004D9903C060E170E002C060E070E0C62BB2
:1021B000D72B4F9903C040E250E002C040E050E00E
:1021C000C42BD52B189903C020E430E002C020E0D6
:1021D00030E0C22BD32B1999A6CF20E830E0A5CF51
:1021E00082E090E0C4CF833081F028F4813099F010
:1021F0008230A1F008958630A9F08730B9F084309C
:10220000D1F4809180008F7D03C0809180008F7712
:1022100080938000089584B58F7702C084B58F7D48
:1022200084BD08958091B0008F7703C08091B00085
:102230008F7D8093B000089590E0FC01E455FE4F3F
:102240002491FC01E054FE4FE491EE23A1F0F0E074
:10225000EE0FFF1FE851FE4FA591B4919FB761119A
:1022600005C0F8948C912095822303C0F8948C913A
:10227000822B8C939FBF08950F931F93CF93DF936F
:102280001F92CDB7DEB7282F30E0F901E856FE4F98
:102290008491F901E455FE4F1491F901E054FE4F89
:1022A00004910023D1F0882319F069839CDF6981B0
:1022B000E02FF0E0EE0FFF1FE252FE4FA591B49128
:1022C0009FB7611105C0F8948C911095812303C0CC
:1022D000F8948C91812B8C939FBF0F90DF91CF91BD
:1022E0001F910F910895CF93DF93282F30E0F901CC
:1022F000E856FE4F8491F901E455FE4FD491F9015F
:10230000E054FE4FC491CC2389F081116CDFEC2F97
:10231000F0E0EE0FFF1FEC52FE4FA591B4912C910F
:102320002D2381E090E021F480E002C080E090E085
:10233000DF91CF9108951F920F920FB60F92112443
:102340002F933F938F939F93AF93BF938091C1013E
:102350009091C201A091C301B091C4013091C0011C
:1023600023E0230F2D3720F40196A11DB11D05C0D8
:1023700026E8230F0296A11DB11D2093C001809372
:10238000C1019093C201A093C301B093C401809195
:10239000C5019091C601A091C701B091C8010196F5
:1023A000A11DB11D8093C5019093C601A093C701E3
:1023B000B093C801BF91AF919F918F913F912F91A1
:1023C0000F900FBE0F901F901895019739F0880F4E
:1023D000991F880F991F02970197F1F70895789434
:1023E00084B5826084BD84B5816084BD85B582601A
:1023F00085BD85B5816085BDEEE6F0E080818160B8
:102400008083E1E8F0E010828081826080838081B7
:1024100081608083E0E8F0E0808181608083E1EB8F
:10242000F0E0808184608083E0EBF0E08081816077
:102430008083EAE7F0E0808184608083808182602D
:102440008083808181608083808180688083109216
:10245000C10008954F925F926F927F92AF92BF92A8
:10246000CF92DF92EF92FF920F931F93CF93DF9360
:10247000CDB7DEB729013A016217730784079507C4
:1024800054F0DC01CB01E816F9060A071B072CF40F
:10249000D801C70102C0DA01C9019C01AD012419AC
:1024A00035094609570989899A89AB89BC89BC01D4
:1024B000CD016A197B098C099D091CD0A8019701DF
:1024C000241935094609570924D02A0D3B1D4C1DF6
:1024D0005D1DCA01B901DF91CF911F910F91FF904E
:1024E000EF90DF90CF90BF90AF907F906F905F9014
:1024F0004F900895DB018F939F932DD0BF91AF91A3
:10250000A29F800D911DA39F900DB29F900D11244D
:102510000895052E97FB16F400940FD057FD05D0B3
:1025200024D007FC02D046F408C050954095309561
:1025300021953F4F4F4F5F4F08959095809570952F
:1025400061957F4F8F4F9F4F0895EE0FFF1F0590AE
:10255000F491E02D09942BD0A59F900DB49F900D80
:10256000A49F800D911D11240895A1E21A2EAA1B8B
:10257000BB1BFD010DC0AA1FBB1FEE1FFF1FA21733
:10258000B307E407F50720F0A21BB30BE40BF50B30
:10259000661F771F881F991F1A9469F760957095B9
:1025A000809590959B01AC01BD01CF010895A29F3C
:1025B000B001B39FC001A39F700D811D1124911D17
:1025C000B29F700D811D1124911D0895F894FFCFC5
:1025D00001000000FF5A0802060804030508000174
:1025E000070808080808212601070000000001016B
:1025F000430001000145005A5A5A5A5A5A014400F0
:10260000010300000000014300005A5A5A5A5A00C0
:00000001FF
